:1000000000308A0080280000603083168F000F08BF
:100010000439043C031D0728831288288316051021
:1000200083120514A630F700F70B1428000083167E
:10003000051083120510A630F700F70B1D280000ED
:10004000003483160510831205145330F700F70BA4
:10005000272883160510831205105330F700F70B7D
:100060002F280034A8012808073C031C4328270830
:100070000139013C031D3E280E203F28212003109A
:10008000A70CA80A3328003427308400000803197D
:1000900058280130F800F701F70B4C28F80B4B28D3
:1000A0004A30F700F70B522800000000800B492867
:1000B0000034FF308316860083120608A600A701CD
:1000C0003220A70132200E205330A70032203530D5
:1000D000A70032202608A70032202508A7003220DA
:1000E00021208316851083128510FA30A700442042
:1000F0008316851083128514FA30A700442000343B
:1001000084011F308305073083169F008312042863
:10011000A1010130A200A300A400831685160030BF
:100120008312851A0130003A031DE2288316051553
:10013000003083120519013022020319AF288316FB
:1001400005158312A2010519A20AA208031DAC28F5
:100150000430A5005920AF280730A5005920831688
:100160008515003083128519013023020319C82830
:10017000831685158312A3018519A30AA308031DFD
:10018000C5280530A5005920C8280830A5005920E9
:100190008316051600308312051A01302402031954
:1001A000E128831605168312A401051AA40AA408DF
:1001B000031DDE280630A5005920E1280930A500DE
:1001C00059202429A108031D112983160515003083
:1001D000831205190130003A031DF4280130A500EF
:1001E00059200130A1001129831685150030831292
:1001F00085190130003A031D03290230A50059205A
:100200000130A10011298316051600308312051A4A
:100210000130003A031D11290330A5005920013097
:10022000A100831605158312051D24298316851543
:100230008312851D2429831605168312051E242981
:0C024000A1016430A70044208D28630059
:02400E00103967
:00000001FF
